:040000000CEF00F011
:0400080021EF0BF0E9
:1000180000EEFFF011EE00F01BEC00F000EEF9F03E
:1000280010EEFFF01BEC00F08BEF0BF0EE6AEA50DD
:0C003800E262FCD7E950E162F9D7120047
:10010000392626262651778C7C85B2DADADADADAD5
:10011000B6856A5A39302C51615651617E93B8D7F1
:10012000DACEA273463B323950666A5D5D5E85AFBA
:10013000DADADABF854626262626395A74877C7491
:10014000747F7F7FA6C8DABF9B68564D6FA0DADA4E
:10015000DADAC97F5A37375E7F9B825E322C2639C6
:1001600068B2DADADACCA67961667994948C735045
:10017000302629488EC8DADABD906650545D686C26
:10018000736A706A6C667987897F73583B26324B35
:100190006C7E7F7F7F7F7F7F7F90A0A69D7C749BFE
:1001A000DADADADAC18C7F7C51392C425448503B80
:1001B0002D295090CEDADADADAB68C7C6A5A546697
:1001C0006C583E2926263977BADADADAC89D705E8D
:1001D000587C7F8579735A39262D426189A2896AB4
:1001E0005D5E5450616C70747E7F7F8582A2ADBF6E
:1001F000907F6F5A506CD3DADADADAB67F7F6C61AF
:100200005A51484D5D462626265A8CD0DADADADA7B
:10021000A693735A5A7C948C8C8C735D5E87978CF2
:10022000745D4D2C2C3F6A8293B2BDA07356504230
:10023000424B6F857F79686A615D616A7074747C16
:100240007F7F7F7F7F7F7F7F85B2DADADADAB67FE2
:100250007F7F7F6A39262626262826263F6C99C866
:10026000DADADADAC18C7F7F74686A737F664626D1
:100270002626265A8EC5DADADAD39B735850565A98
:1002800068634D37292C3946617C9BA6A2907C730C
:100290006A6A747C85826F5A546C7F7F7F7F7F7F10
:1002A00085C8DADADADAA67F7F7F7F7F5A3E262694
:1002B000262626264B7497CCDADADADADAB67F7F8E
:1002C0007F7E6661686F583E3937303E638CA4B8D4
:1002D000CCCCB3948789878577745E4626262626FC
:1002E00035568597A2A69D8C77746F797F7F7C6841
:1002F000685A6C737F7F7F7F7F85C8DADADADAB677
:100300007F7F7F7F7C563E2C3729262626294B6C03
:10031000ADD3DADADADACCA08C7C7373858E896C93
:100320005A2C262626426C93AFC4C5BAA69B897E5A
:100330008590997F74563F2626263E5E778C939053
:10034000877E7973707C9393796658565A6C7F7F59
:100350007F7F7F7F97DADADADADAA07F7F7F7F7FAD
:1003600066502626262626263F486C9BC8DADADA0F
:10037000DADAC1A28C7E6A5458707C5E563E292619
:10038000263E5887A9CEDADAC5B2A08E777F796F7C
:100390005D56392D263B3F636F8E97A99494897FD4
:1003A0007070747777796F685D5A61737F7F7F852E
:1003B000DADADADADAB67F7F7F7F705650545E443D
:1003C00026262626264B7E9BC8DADADADAD7B2A2B0
:1003D0009790857F7F7C664426262626264D749737
:1003E000ADBAC1B6C5BAC1AFA497857463483B2CFA
:1003F000303748586F77878E8E8E85877E7C7C82DB
:1004000094949073684D484861749BDADADADADACA
:10041000B67F7F7F7C5A442C39504846292C2629A8
:100420004B7F7F7FB2DADADADADAC4AF9D908C855F
:10043000857F735A30262626264B6387A4C1B6C90A
:10044000BDC8A6A6949782776A5D54463F373E445E
:10045000565E79899799978E938C897E7F82857F66
:10046000735D5648515D87BFDADADADADAB68C7F27
:100470006C503937444D4D48423729263F617C7FC7
:1004800085AFDADADADADAC5B6ABA097908C7F748A
:100490005E442826262C48667FA2ABB6B2B2A09353
:1004A000897E7F77797F897E7061504646565E6F80
:1004B0008797A4A2A49993827E736F6A6861515151
:1004C0003E4D5077A2C4DADADADAC9A4855D463B3C
:1004D000374256636F6A5E513F3E4B687F85A6C8C0
:1004E000DADADADADAD7CCA28C7F7F7F7E68503016
:1004F000262D3046507487939094939D9BA2949799
:100500008E9D97A0897C665A58585D63707C909444
:10051000948C7C68565061566361776F5D484B617F
:10052000749BB2DADADADADAA67F5D48504861778E
:100530008E93745E4B423F303F507797ADCED7D706
:10054000CCBFC1ABADA6ADA0A29389705D443E35D2
:100550003B3E586A798E94939497948C7F8E8C9BB3
:100560009B9B97827468635D5154616C7C6C706373
:10057000615D617374746C615D5A6A747FABC4DAD7
:10058000DADAD5A27C6C686166778E9489827768A6
:10059000564844545E5E7C8EA2A2A0999493909D8E
:1005A000ADC1C1CCC5B6997E66503B373E56687723
:1005B0007C7C7F7C635D5066688993A6B2BAAF9BF2
:1005C000897E746C6F737C7C828287857E665E56C2
:1005D000635E70777E6F5E544D484B617494B2DAFF
:1005E000DADADABD9985747070909BADA6A4907725
:1005F000563E30353E54687F90908C7F7F7E7F875B
:1006000090B2BAC8C5B8AD8C7E63545A616A6F6F38
:10061000736C5E504B56636A829DB2C1BFB29B89B8
:10062000776A637077878C908779705E6363777E73
:1006300085898E8E827E6C685D5A5E667370747F6B
:1006400087878E979B9D979D9BB2ABAFA29D938909
:1006500089877E77686C6A70706F70666A6A707F6F
:100660007C8E85A49BA68E8C8987897F827E746F01
:100670006A5D666C79706F747F85878C8C877C7FF0
:100680008594909382827C7F707F737E747C797F67
:10069000777F73857C857F85827C827E857E797776
:1006A000797F7C737370777F7F8C82908793908E35
:1006B000878597939B8C9482877F827770777E7CE7
:1006C0007F7E7C797F85828587897F827F7C777436
:1006D0006A7E7E7F70747E7E7C7E7E777E7E8C825C
:1006E000877E857E7F7E7F85827E7E828279777718
:1006F000857F7F7C7F857F7C79827F827F897F7EFB
:100700007F89827F7C828287857F7F7F7E7F7F82D9
:100710007F8C7C79707F87858279797F8282827FE6
:100720007F7E8590857F747F8E8C7E85738E7C7FA7
:10073000747F8E8E7F7370748E7F8C7F7F827F82BA
:100740007E747F747F7F7C7E7E827F7F7F7E7C7CD9
:100750007C7F798593877C7385877F8E8282737F88
:100760007E7F7F7F7E7E82827E7C8282827F827E8F
:100770007E7E857F7F7F827F7E7F8E7F797382877B
:100780007F7E7E8E7F7F737F8E7F8E737E737F8270
:100790007F8E827F707C82857E7E8E938E7F7F743B
:1007A0007E738C737F747E7F7F827F7F7E7F7E856A
:1007B0007F7F7E7E7F82827F8C7E8274827E7E7F40
:1007C0007E7F7E7F82857E7E7F827E7F7E827F852A
:1007D0007E7C827F857C827C857C827F877E7E7C1E
:1007E0007F827F827C857E7F777F7F858282827C0D
:1007F0007F82827F7F827F7F82828C8C7E73747FF8
:100800007E7F7F857F7F7C7E7C7E7F7F857E877FEE
:10081000827F7E7F7F857F8C7F82737E7E7F7F7EDF
:100820007F7C7F82877E7E7F82797F7E857F827FCD
:100830007C857E857C857C857E827F827F7E827CB6
:100840008279857C827C7F777E7F89827F827F7CB4
:100850007E8587857F827E827E7F8C7F7E737F828E
:10086000827E7C7C7F7F7F7E827F7F7F7F877F858C
:100870007F827C7C7F7F827C827E7F7C82877E7E83
:100880007C8282827F797E7E8285857E7C7C858269
:10089000897F7F7F7F7E7F82857F7F7C7E827E8255
:1008A0007C857C857E7F7C7C7F7F828290857E7349
:1008B0007F908E7F7473827E7F8C7F7E707F828537
:1008C0007F7C7C827F827F827E7F7F7F7F7E7F7F37
:1008D00082827C857E857F7F7C7F7E827F827E7E1A
:1008E000857F7E7C85827F7F7F7E7E7C877F858CF7
:1008F0007C7E7385827F8E827F73797C7E7F857F0D
:100900007F797F7E828585827E857F7E7E85827FE0
:100910007F7F997F7063739D87856F7E947F7C6CEA
:100920007F7F87827F827E7E7C7F7C7F85897F7EC2
:100930007F85857E7C7E85827F7F827E7E7C7F82B6
:10094000857E7F7F7F7F7FBF82503B9BD379506FB7
:10095000A0A26373828C826F7F7F82CC7F51308CA8
:10096000C8735E8CCC824846A497666F8E97796672
:10097000827F8977B693684BA2C997516CA07F5A42
:10098000547EA67F6C9D7F734D90B26A6F739B827D
:100990007EA09D975A61A0746679B87F265AD5D5F6
:1009A00056469DAD5A4D94A97C6A94977363829084
:1009B0007C7CA4AB875A737F5D4D73D5B889748EE8
:1009C00085374899A67066997F6866A6936F7C897B
:1009D0007F617EA9947FA0A4997990875446617322
:1009E000857E8CA69D74665A7C61858CA0948782D6
:1009F000A4C9937F77AB6F2D77778C426A87737426
:100A00006C9B8E777F7F997E9B997F7F7FA9737C7C
:100A10007973685E776F7785998E707F7F6C6C795C
:100A20009B85799DA2996F878C936A5D5E637374D1
:100A30007089879777898E8985637C7F897C6F89A8
:100A40007E777E747C637F74707C8C8C6F7C908EE0
:100A5000908C85746C898285877F8974827E857F7E
:100A60007F7F7F897F7F8C908E7C907C87748E7E49
:100A700087797F828785878CA28C8E879989897FE9
:100A8000878779826F877C7E7F777E708C7F828775
:100A90007F778297827779947E737F857F7E908738
:100AA0006F7E8E876F798E7F705D7C7F7F6A6A9B99
:100AB00090937C979482777E828279827E797C89FA
:100AC0008974778E8E7466908C85667F9087747932
:100AD0008285737F7F877F89858985897989877EEC
:100AE0006F79857C79878973737F897E737F7C7C3E
:100AF0007F937F668297825A738E826C6C907F6C34
:100B00006C7F7F686385827466747F897F777C7F62
:100B10008C747E829B8C878289828C7E7F7F878784
:100B200079ABB8AF879DB2A48E93A69D897F7C8256
:100B3000777F7973706A706F746F6F6F7070778979
:100B40008777777379737C7C686668706873747E66
:100B5000797974777F8C8C7C6C7E8E736A737C87DA
:100B60008C6F54709785667F7F5D6C9397566AAFE4
:100B7000DABD99A6D5C5AF97938C97856F4B7C6FDF
:100B80006F3751637E737C828EA9B3AFA2A9B694EE
:100B9000796F7F6A5D445D615E545E6F74707370DF
:100BA0008787907F777F7F82797F7E7E6A685E63AA
:100BB0006A63686A7079828297A08E74829B8C6A5D
:100BC0006A746C6674CCDAC49DC1DADAA98EA6A602
:100BD000907C70666F6A633E29667E824B5D7C9B6B
:100BE00094A0A6C4DADA997F85A96A463F5A5D487F
:100BF00044465D70827C747F908E7E7E7E9385738A
:100C000063737F6A54515E5A5A66746F74877F7F2C
:100C1000899D7E707FA097796F7070738CDACCB6E7
:100C200085DADAD79799B2906A5E5E68615E504B5A
:100C3000617770636A8C949793A2909B99A2A4C1E8
:100C4000BD73567F9D63263763664D5879909494A3
:100C5000826C8290875D5A6C6C63616170666C63B4
:100C60006A706F73747F6C79829B878787856C66E7
:100C70006A74D3DADA9399DADAA66C82A6876648C0
:100C80003B3E5A7039284693A0797C97BFB3B699FA
:100C90009390A9A6907E7782907951446C74663FB8
:100CA0006A859982798589947E6F546163665D5601
:100CB0005E6168616C6C8270746C7C8C9079666625
:100CC0009D8970507082A6DADAD07FDADADA797428
:100CD0007F995A46263E3E615044357EA6A68599A8
:100CE000C1D0B8A29B8E8C8987795D637C8C6F4B59
:100CF0005A7F8973667F97977F7E74877F73564884
:100D00005A63665156666F6F6F7070797C7E707F24
:100D1000877473878268567E7F7E70DADADA50D302
:100D2000DADA777F7F855650262626566F4435823D
:100D3000C8C9A2ABC9D3C4AB9B74777C8563445844
:100D4000748974616F7F94827774949B8C6C667CD9
:100D5000776A5151565D5D565E707E6A58666F7C4B
:100D60007F8E7F6A7C7F7E636A777C7F97DADAC8C2
:100D700050D3DADA73747F795A392626267073488D
:100D80003787D3DAC8B2C4CCCEAB906368747F51D6
:100D9000394B7087797977899DA487737997875EB6
:100DA000516A7C66544B585E66615D5E7377745E13
:100DB00079907F5A66A28C664B777F7F7EDADADA8B
:100DC0007FA6DADA87747F6F503E2626263F82633D
:100DD0003F6FD3DAD3BAC8CCBAAB946F48617F66A1
:100DE0003237799D876C7090A2AB8C797493856350
:100DF00050617C68443F506C6F68685A707E856AA9
:100E00006368737F747366747F7F7F7FDADADA7F5B
:100E10007FDADAB670705E54482D26262C999463DA
:100E200063BDDADAC8ADB2C1C1935A35516F6F3FB5
:100E3000305D90B2A9877E93B89D6354778C6F50D4
:100E400056616C635E46516A7F6C505A7387736358
:100E500066777374707F7F7F7F85DADADA7FC8DA2E
:100E6000DA7C666C544B2D2626266FAD7C5A7CDAD4
:100E7000DADAB6ADB8B3A6682D3561794D37468C50
:100E8000A9B69B8C90A9B38C5D51707C5A3F3F6A88
:100E90007E706156637074685056777E745E616FC1
:100EA000737F7C7F7F7FB2DADAD597DADACC6C6633
:100EB00061513E2626262887A2796ABADADADAB69E
:100EC000ADB2AD9B5A262666703E2850AFCCC8996D
:100ED0008EA2BFA06F3E50666F4D3F516F7E6C5A21
:100EE00056748777515173746A50616C7C7F7F7F31
:100EF0007F7FDADADA9DA6DADA8C6A6A3939262651
:100F0000262650A9A67F97DADADAC8B3A2A4996F89
:100F100026263F705E323F7EDADAC48C8EBDB26F19
:100F200032376A6C54395070857C5D48617C7F56DD
:100F30004D5E85795E56687F7F7F7F7FDADADAA241
:100F40007FDADAB65A5A3942322626264DBAB285A7
:100F500085C8DADADAAB909B9D7732263F6A703B20
:100F60004D9BD3D7AF97999DA6744D44616F514463
:100F7000507079736856636F7451485E7F7E615E0E
:100F80006A7F7F7F7FDADADAC47FDADAB6685A39C5
:100F900026292626262D93B69B97C8DADADAB39D42
:100FA0008C896C37262C616C4B56ABD5DAB3A09785
:100FB0009D97734D46566A6354566C7970615D5EB9
:100FC000686A5A5456666C6F74747C7F7FB2DADA42
:100FD000DAB2C8DADA68543E3B353226262682B8C1
:100FE0009785BDDADADAB89493897C482626617F42
:100FF00066507EC1D7D0B3948C90935E37426677AB
:10100000564D5A748274635666736A544D586668B6
:1010100073747F7F7FDADADAC48CDADAB65A503941
:10102000393026262644ADB39393DADADACCAB8C8A
:10103000908763282632707E615D8ED0DAC89989E8
:10104000949B70513E636F6351586C77746C585D1C
:101050006A706A505D5873737373747FDADADACC2E
:10106000A2DADAC15A50393F3B2626263B9DAD9382
:1010700087BDDADADAA68E82907C3E26266C7F6CFB
:10108000567EBFDAC89D8589A07F5630567370544E
:10109000506A7F856F58587470634B5E666A616CE6
:1010A000747F7FB2DADADAA2DADAC15A4B39483B16
:1010B0002626263B93B29793B8DADADAA689858595
:1010C000743726296377797089ADD5C59B7F909356
:1010D00073544D6170635E566C7C826C5A5D6A6AB3
:1010E0005A54616C6C5E68747F85DADADAC9ADDAFD
:1010F000DAB3664430353F2D26264DA2A68987B641
:10110000DADADAAB93857F6A372629616F797E90C8
:10111000AFBFC8AF8C7F7F73584D5E6F63616373E1
:10112000747F7763585E736A615E5A5E6677747027
:1011300074B2DADADAB2B3DADA90463932543726F0
:1011400026267FB8A087A6DADADAAD8E8C947E4D9B
:1011500026264B776C5E87C1D0BDABA9947F7466A1
:10116000464D6679615A6C857F7E685D516A6A6317
:1011700050586666706674747F9BDADADAB2B8DA51
:10118000DA9051443E422C2626266AADA07F9BDA97
:10119000DADAB89D93907E5129264458615D77A490
:1011A000CCD5C8ABA297875E515061685D5E5E7E0C
:1011B000878E7066636C745E58566F6F56515873A5
:1011C000747E7FA6DADADAB2CEDADA8751443242B6
:1011D0002C2626266CAB9D89A9DADADABD99949380
:1011E0008254262639505D566690CEDAC494A4BF48
:1011F000B26F4D5466614D4D5A7E898E74707C7FFE
:1012000073545D6A736A505A5D665A61747F7FA633
:10121000DADADABAC4DADA9B54483E3F28262626C0
:101220005E979B879BDADADAB8A2A0947E563B2CB5
:101230003B463E394D90B6C1C8CCD0C4B89D6F5422
:101240005A5E463544738587827C7E7C82685E5E0A
:10125000746F635E5A6A6A615056737F7F9BDADAF5
:10126000DAB8AFDADAB25A4842483226262656971A
:10127000977993CCDADAC8A4ABAB8C633E323F4D9E
:101280003F2C3F7097B2B6DADAC8AFC8B2794B5E7E
:10129000543E28465D73798285899D997C616C797D
:1012A0006A5D636F6F66635656565E68747F85C865
:1012B000DADADAC4DADAD0775A5451372626263207
:1012C0006A7F7374B6DADAC8ABC4C5B27958424BD8
:1012D0004D4826264679907CABDADAD7A6A6BDAD76
:1012E0007744424B51483F4B6C8E878282A0A29339
:1012F000736F6C79706C616A6A6F58515666635A85
:1013000061737F85B2DADADADADAD5DAB25D504DB6
:10131000482626263251707F7C9DC1DADAC8BABDD4
:10132000B89B775D42423F35293556747F87A2BD11
:10133000DAC9DABDBA9979684B4D4B5454545E6C96
:101340007E8582939B9D93857F82878270666C7079
:10135000706A68616A6A6C6A6A636F796F5D567CED
:10136000A6C4DADADAB2B8DADA905174795D2C26EA
:101370003944585D686694BDC4A29DC5D7B68974CA
:10138000797366543F3B506366566A94ABA0B8C409
:10139000D3AFA29B977461585D5A48565A666C7CCD
:1013A0008789878E909085937F8E7E8C746F6C700A
:1013B000736C686C7074777C827F7E79736C635A0F
:1013C000687093BDDAD394ABDADA9B5D77977C468D
:1013D000283746505A50517FB2AF8C8CC1DABA8C44
:1013E0008799937963515861664D445D798C7F7F0D
:1013F00094A2AF999D999D937F706F7E7961566895
:101400009085746C82898574827E8C82857F9097AA
:101410009070686F77737074746F6F777F7F7F7E63
:101420007F7F827E6F686A7470707FABCCD0897F5B
:10143000C4DACC707CA2945D42505D544D4B4D6A31
:101440008C907985A2C9AFA093A6A48C746A73709E
:101450007054505D7770637390A2938C9999A690A5
:1014600097877F89827E6A7073635D5D7077797C10
:1014700079859093937F938E82737E7E7768707464
:1014800070776F747079827F877E85747474797CCD
:10149000747985B2CEA07EABDAC87974A09B795DF1
:1014A0005E6A6F68504B5687796F738EA4978C94E1
:1014B000A9A69487898C8E7E6F61707763585E7C55
:1014C0007E77748290908985939D9D8E8990898284
:1014D000797F77706863686674707E7C85828589A1
:1014E0008E8E7F7F7C8779776F77777E7779777E2F
:1014F000777779897E77747F8577777F7E85A6C1B8
:10150000897FADD7AD7393AD94746873737466546B
:1015100046667F6C5D63939489859DA49B908E8CB9
:10152000939082777E7970636F6C7E686C6C7F8736
:101530007F7F8E999D8E7F94948E79798577705E6A
:101540006C6C7370777C827F827E8987897C7F82D6
:101550008E827C6F77737C79827C73777F87797ECC
:10156000797E7487896F6C87937F7CB3B28973AD02
:10157000AFA07F9D93827E7F74737C7056667C7E65
:10158000616A7E7E797C908C899793948993877F1A
:10159000797F7F7E7C777C746C6C737F7C7E7F82AE
:1015A000827F93908C85878E7F7C77857F7C74701B
:1015B000746A7973827E7F777F85877F857F7F7C62
:1015C0007F797F7C827479777F7E7C7E7C7E797F59
:1015D000877974797F7F778E99937F8CA29397898F
:1015E000A6858589939079796F7F797E7073796C00
:1015F0006F6F8C827F737F827F908E8285828E7FD9
:101600007F877F7F7F7F7C77797F747F737E709306
:081610008E7F7E898E7F790038
:10161800F29EF20ED36EF70E936E7F0EC16ECA6AFB
:10162800B50ECB6E9E929D82CA840C0EBD6EBE6AAC
:10163800BD9ABD98F28CF28E12009EA21100000194
:10164800F951FA11D8B403D0F907000EFA5B9E924B
:101658001100F3D7D96ED9CF00F0D8900032D890C6
:101668000030BE6ED9CF00F0020E0016010E016EDA
:10167800D8900032012EFCD70030BD9AD8B0BD8A70
:10168800D9CF00F0016ABD9800B0BD881200FB00F8
:10169800F36AF46A0001F450800A006EFE51800A71
:1016A800005C02E1FD51F35CD8B01200FBC000F011
:1016B800FCC001F0F3500026F450012200C0F6FFF0
:1016C80001C0F7FF000EF76403D00800F55005D0FD
:1016D800F6CFE9FFF7CFEAFFEF50BCDF0001010EBC
:1016E800F96FFA6B0001F951FA11D8A4FBD7F34A44
:1016F800F42AD0D7FB00000EADDFFBC0F9F0FCC028
:10170800FAF00001F951FA11D8B41200FAD780DFC3
:101718000001010EF96FFA6B0001F951FA11D8A412
:10172800FBD70001000EFB6F010EFC6F170EFD6F5B
:10173800150EFE6FADDF0001FB6B7D0EFC6FDBDF6E
:02174800E7D7E1
:020000040030CA
:04000000FF38FCFECB
:02000600FBFFFE
:020000040000FA
:00000001FF
